:020000040000FA
:06000000D1EF06F0120032
:0600080004EF08F01200F5
:060018000CEF08F01200DD
:02001E001DEED5
:0E00200000F02DEE00F0F86AEDEF06F0120091
:020030000000CE
:0E0032003E0E126E136AFC0E146E156A166AEC
:1000400019681A681B68186A1200D9CFE6FFE1CF59
:10005000D9FFE65216501EE1040108BF1AD0400E27
:10006000E66E600EE66E000EE66E95EC06F0E5526A
:10007000E552E552010E166EDF6A400EDF5C09E2C2
:10008000DF50EA6AA00FE96E000EEA22EF6ADF2A6B
:10009000F4D717D100016051080A01E10DD10F0A10
:1000A00001E1D3D0010A01E1CAD0030A67E0010AE5
:1000B00058E0070A44E0010A01E003D10001020E02
:1000C000A06F00013A0EA16F0001010EA26F0001A6
:1000D000010EA36F0001A46B100EA56FA66BA76B9A
:1000E00013C0A8F014C0A9F015C0AAF0100E0001AA
:1000F000A95F000E0001AA5B0001AB6B0001030EBB
:10010000AC6F0001F80EAD6FAE69AF6BB06B000164
:10011000080EB16FB26BB36BB46B0001B56904012B
:100120000CBF0CD0400EE66EA00EE66E000EE66E22
:100130005BEC06F0E552E552E552166AC2D00001CA
:10014000615107E13F0E126EF80E136E1468156AC6
:1001500006D03E0E126E136AFC0E146E156A166AF5
:10016000B0D0040E176E1228175C06E20400AED859
:10017000F0EC04F0172AF7D7166AA3D0E86819182C
:1001800005E1E8681A1802E1E8681B1806E161C099
:1001900019F062C01AF063C01BF019500001611918
:1001A00008E11A500001621904E11B5000016319B3
:1001B00000E143E1DF6A00016551DF5C3EE2000ED1
:1001C000195C100E1A58000E1B582CE312285C6E96
:1001D0005D6A0A0ED8905C365D36E806FBE15E6A21
:1001E0005DBE5E685C50195C5D501A585E501B58CD
:1001F00019E23A0E0001D8806555DF24EA6A660FDD
:10020000E96E000EEA22EF50E66E1850E96EEA6AD7
:10021000E9BEEA681C0EE926000EEA22E552E75024
:10022000EF6E182A192A000E1A22000E1B223A0E0F
:10023000185C01E15ED8DF2ABED7166A42D059D8D1
:1002400019681A681B68166A3CD00001070EA06F77
:1002500061C0A1F062C0A2F063C0A3F064C0A4F0CA
:1002600065C0A5F061C0F6FF62C0F7FF63C0F8FF8C
:10027000DF6A00016551DF5C0FE209003A0E000100
:10028000D8806555DF24EA6AA60FE96E000EEA22DF
:10029000F5CFEFFFDF2AEDD704010CBF0CD0400EE5
:1002A000E66EA00EE66E000EE66E5BEC06F0E55222
:1002B000E552E552166A05D06592656A68D8FF0076
:1002C00000D0E552E552E7CFD9FF1200F66A175089
:1002D000F76EF86AD890F736F836F736F836140E17
:1002E000A66EF29E550EA76EAA0EA76EA682A694C3
:1002F0001200D9CFE6FFE1CFD9FFE652DF6A000E48
:10030000E76E1818E8AE02D0183403D0E750D88052
:10031000185436E218505C6E5D6A5E6A5CAE02D0BC
:100320005D685E685C50195CF66E5D501A58F76E39
:100330005E501B58F86EDF50EA6A1C0FE96E000E23
:10034000EA22EF50F56E0D00DF2A1806185009E07A
:10035000DF50EA6A1C0FE96E000EEA22EF50F56EDC
:1003600001D0F5680C00DF2A240EA66EF29E550E11
:10037000A76EAA0EA76EA682185001E01806BFD776
:10038000A694186AE552E552E7CFD9FF1200D9CFFB
:10039000E6FFE1CFD9FFE652DF6AFF0EDF5C0AE23B
:1003A000E868E85005E0E80600D000D000D0F9D7B2
:0E03B000DF2AF3D7E552E552E7CFD9FF12005E
:0203BE00D9CF95
:1003C000E6FFE1CFD9FFE652645032E162960401C4
:1003D00000513C0BE842E8420D0828E1180E0219D2
:1003E00023E1040E031920E1100E026F040E036FC7
:1003F000DF6ADF505C6E5D6A080E5C5C000E5D5863
:1004000013E2DF50EA6A180FE96E040EEA22EF5099
:10041000E66EDF50EA6A100FE96E040EEA22E5523A
:10042000E750EF6EDF2AE5D711D80AD046D808D0BA
:10043000040E645C03E162965CD802D0000E01D029
:10044000010EE552E552E7CFD9FF1200D9CFE6FF02
:10045000E1CFD9FFE652040104BF046B0C6A086ABD
:10046000096A0A6A0B6A87EC03F0DF6ADF505C6E88
:100470005D6A010E5C5C000E5D5819E2095017E1DF
:10048000F76ADF34FE0BF736F66E5A0EF6260F0EBD
:10049000F7220900F5CF5CF00800F5CF5DF004D03D
:1004A0005DC0FAFF5C50F96EFBDFDF2ADFD7EDD8C5
:1004B000E552E552E7CFD9FF1200020E085C0EE1CB
:1004C000A7D80401180E026F040E036F080E016F07
:1004D00000BD02D0C80E0BD0880E09D014D904017B
:1004E000080E016F100E026F040E036F8C0E006F6A
:1004F0001200040E0E5C0AE112C438FF0F013851DD
:10050000000802E2050E01D0030E0E6E08040FE192
:1005100010D8020E0C5C03E10401840E06D0040125
:1005200004BD02D0C80E01D0880E046F120083EF04
:1005300003F0D9CFE6FFE1CFD9FF020EE126080E86
:100540000A5C000E0B580DE20AC0DEFF0BC0DDFF97
:100550000C5002E1010E03D00C0406E1020E0C6EF9
:1005600003D0080EDE6EDD6A040104930491010ECF
:10057000DB500413DFCF05F4DE500A5EDD500B5A6A
:100580000001180EE26F040EE36F0FA21CD0D9CF4A
:10059000E9FFDACFEAFFEE50ED1030E0E0C0F6FF01
:1005A000E1C0F7FF0800F550E2C0E9FFE3C0EAFF51
:1005B000EF6EE22B000EE323E02BE123DF06010EBA
:1005C000E6E2DB06E4D7D9CFE9FFDACFEAFFEE5067
:1005D000ED1014E0E0C0E9FFE1C0EAFFEF50E2C037
:1005E000E9FFE3C0EAFFEF6EE22B000EE323E02B0E
:1005F000E123DF06010EE7E2DB06E5D7020EE15C50
:1006000002E2E16AE552E16EE552E7CFD9FF12005E
:10061000D9CFE6FFE1CFD9FF020EE126030E040198
:100620000015E76E010EE7CFDBFF01C4DFFFDE50F0
:100630000A26DD500B220001180EE06F040EE16F58
:10064000D9CFE9FFDACFEAFFEE50ED1014E0E0C0B9
:10065000E9FFE1C0EAFFEF50E2C0E9FFE3C0EAFFD3
:10066000EF6EE22B000EE323E02BE123DF06010E09
:10067000E7E2DB06E5D7020EE15C02E2E16AE55261
:10068000E16EE552E7CFD9FF1200659809500BE102
:100690000401080E016F100E026F040E036F840E2A
:1006A000006F04011ED0040110AF1DD00A50165D6A
:1006B0000B50175904E216C40AF017C40BF039DFC7
:1006C000010E086E0401080E016F100E026F040E79
:1006D000036F800E006F0401180E066F040E076F83
:1006E000C80E046F1200020E086E0401056BC80EDE
:1006F000046F0401080E016F180E026F040E036FE1
:0E070000C80E006F1200086A0401046B12009C
:02070E000401E4
:100710001051600BE842E842E842E842E842000932
:1007200001E012001151070A43E00B0A41E0070AF9
:1007300034E0010A24E00B0A20E0020A1EE0030A6A
:100740001AE0080A10E0010A0CE00F0A08E0030AA8
:1007500001E01200010E096E040E0E6E1200D9EFB8
:1007600003F029EF04F0010E096E0001100EE06F96
:10077000000EE16F0ED04DEF04F08EEF04F0010E8D
:10078000096E14510001E06FE16B110EE027000EBD
:10079000E1230F92010E0A6E1200010E096E145130
:1007A000EA6A110FE96E000EEA2212C4EFFF12008E
:1007B0001200800E0401105D4BE11351030A2DE07D
:1007C000010A0BE0030A43E1010E096E00019A0ED3
:1007D000E06F0E0EE16F120E38D0010E096E12514D
:1007E000F66EF76AD890F636F736500EF6260F0EEC
:1007F000F7220900F5CFE0F00A00F5CFE1F0020E94
:100800000001F76AE025F66EE151F7220900F5CF05
:100810000AF00A00F5CF0BF01AD0010E096E125142
:10082000F66EF76AD890F636F736540EF6260F0EA7
:10083000F7220900F5CFE0F00A00F5CFE1F0E0C0C3
:10084000F6FFE1C0F7FF0800F5500A6E0B6A0F8251
:100850001200010E096E0F0EE66E270EE66E0F0EE9
:10086000E66EC9EC05F0E552E552E552010EE66E82
:10087000110EE66E000EE66EC9EC05F0E552E5528B
:10088000E55212C410F00401125103E1050E0E6E80
:100890001200060E0E6E46EF06F00401186B196B7F
:1008A000040110511F0B020A0EE0030A09E0010ABD
:1008B0002AE1010E096E0FA026D00401188323D06F
:1008C000010E096E20D0010E096E14510F0B080D98
:1008D000F3505D6A000F5C6E040E5D221451800BB4
:1008E00001E0010E040DF35000015C24E26F000EE4
:1008F0005D20E36FE2C0E9FFEA6EEF50040B03E016
:100900000401010E186F090408E10001180EE06FE0
:10091000040EE16F0F92020E0A6E1200040112051E
:100920000CE110511F0B000908E1010E096E030EC6
:10093000115D02E10F8001D00F90125134E110518E
:100940001F0B020830E114510F0B00092CE0010EBF
:10095000096E14510F0B080DF3505D6A000F5C6EA9
:10096000040E5D221451800B01E0010E040DF350C2
:1009700000015C24E26F000E5D20E36F030E0401B2
:10098000115D02E1840E03D014AF07D0400EE2C027
:10099000E9FFE3C0EAFFEF6E1200880EE2C0E9FF54
:0809A000E3C0EAFFEF6E120054
:0809A80065A60CD80E0409E15C
:1009B00065BA07D0626A0F01366B36813689020E3E
:1009C0000E6E1200656A0F01366B6586010E0E6EA3
:1009D0001200656A0F01366B0E6A1200E9EF04F02F
:1009E0000E5001E112006250040B05E00F01365178
:1009F000040B01E083D865B212006250010B05E0E0
:100A00000F013651010B01E093D86250100B05E045
:100A10000F013651100B01E01FD86250200B05E08A
:100A20000F013651200B01E071D8030E0E5C01E27C
:100A300012000D6A040E0D5C0EE26250080B0BE012
:100A40000F013651080B07E0DFEC01F0000901E16E
:100A500062960D2AEFD71200D9CFE6FFE1CFD9FF7A
:100A6000020EE12636CFDFFF0F01040E366F6298CB
:100A700065828C50040B01E0010E5C6E8C50080BFB
:100A800001E0010E5C10E76E010EE7CFDBFF8C96F4
:100A90008C94A198A0880300A150100B05E1D050C0
:100AA000080B02E10300F8D7A098DF500F013613BE
:100AB000010EDB50E8B08C86E8A08C96010EDB506E
:100AC000E8B08C84E8A08C94D50E056E020E066EFC
:100AD00005C05CF006C05DF00506000E065A5C50CD
:100AE0005D1002E00400F4D7020EE15C02E2E16A6C
:100AF000E552E16EE552E7CFD9FF120065920F0192
:100B0000369562A402D06294FCD712000F0126A190
:100B10000DD0800E0401005D07E1840E0401045D28
:100B200003E104018C0E006F0F012691629A1200FE
:100B3000636A626A0F019F0E376F0F017B0E366F7B
:100B40000F01386B0F0EE66E270EE66E0F0EE66E87
:100B500020D8E552E552E5520F01160E266F62A627
:100B600005D0629600D000D00000F9D7659883ECDC
:100B700003F00401080E016F0401100E026F040E51
:100B8000036F04018C0E006F0F90106A030E0E6E3F
:100B90001200D9CFE6FFE1CFD9FFFD0EDBCFE9FF91
:100BA000FE0EDBCFEAFFFC0EDB5004E0EE6AFC0E2B
:0C0BB000DB06F9D7E552E7CFD9FF1200B1
:040BBC0004011051CF
:100BC0001F0B010801E01200145101E01200060E93
:100BD000115D21E11351230A1DE0010A0DE0030A12
:100BE00019E1020E096E100405E10001BE0EE06F6E
:100BF0000E0EE16F090E0CD0020E096E100405E115
:100C00000001330EE06F0F0EE16F100403E11D0EC3
:100C10000A6E0B6A0F8204011051600BE842E84231
:100C2000E842E842E842010801E0120011510B0AD3
:100C300026E0080A19E0090A12E0080A09E00B0A8E
:100C400005E0080A01E0120044EF06F045EF06F067
:100C5000020E096E0001000EE06F000E0BD0020EB6
:100C6000096E13C400F01200020E096E0001010E9D
:100C7000E06F000EE16F0F92010E0A6E1200020E7D
:100C8000096E12C401F0120012001200026A0F0174
:100C90001E0E276F0401400E096F200E0A6F040E0E
:100CA0000B6F880E086F0401600E0E6F040E0F6F3D
:100CB000400E0C6F1200D9CFE6FFE1CFD9FFE6520C
:100CC000FC0EDB50400805E2400EF36EFC0EF3CF45
:100CD000DBFFDF6AFC0EDB50DF5C19E2DF50E76E02
:100CE000FD0EDBCFE9FFFE0EDBCFEAFFE750E92682
:100CF000000EEA22EF50E66EDF50EA6A600FE96EFE
:100D0000040EEA22E552E750EF6EDF2AE3D7FC0E2D
:100D1000DBCF0DF4400E04010C170C7D880E0C1374
:100D2000E552E552E7CFD9FF1200D9CFE6FFE1CF78
:100D3000D9FF026A040108BF2FD0FC0EDBCF5CF0A4
:100D40000951D8805C5403E2FC0E09C4DBFF026A3F
:100D5000FC0EDB50025C19E20250EA6A200FE96ED9
:100D6000040EEA22EF50E66E0250E76EFD0EDBCF76
:100D7000E9FFFE0EDBCFEAFFE750E926000EEA228C
:100D8000E552E750EF6E022AE3D70401400E096FE7
:100D90000817087D880E08130250E552E7CFD9FFE7
:020DA00012003F
:0E0DA2001DEE00F02DEE00F0F86AF66A100E5D
:100DB000F76E0800F550FF0808E1010EF66E100E00
:100DC000F76E0800F550FF0806E080AE02D000EF95
:100DD00008F080AEFED701D812000DD8040034D838
:100DE00037D8060E0E5C05E16550020B02E125ECDA
:100DF00000F0F4D71200600ED36E9B8C580E056E77
:100E0000020E066E05C05CF006C05DF00506000E21
:100E1000065A5C505D10F6E165A604D06592656ADD
:100E2000C7EC01F00F01140E396F0E6A0F6A106AD9
:100E300019EC00F0036A046A8C968C94959695944C
:100E40000F01486B496B1200D4EC04F0F0EF04F092
:100E50000350041004E1100E036E270E046E030607
:100E6000000E045A060E0E5C02E28C868C94060E6E
:100E70000E5C12E1035004100FE10001075102E182
:100E80008C868C94030E075D02E18C968C84072B74
:0A0E90000751030801E2076B12008E
:060E9A001201000200003D
:100EA0000008D8043C0002000102000109022900E8
:100EB000010100C032090400000203000000092102
:100EC00011010001221D00070581034000010705F3
:100ED00001034000010403090434034D0069006369
:100EE0000072006F00630068006900700020005409
:100EF000006500630068006E006F006C006F0067A3
:100F0000007900200049006E0063002E002603488F
:100F100000490044002000550053004200200042D8
:100F2000006F006F0074006C006F0061006400656A
:100F30000072000600FF0901A101190129401500F6
:100F400026FF00750895408100190129409100C0D5
:0C0F5000AC0EAC0ED50ED90E0D0FBC0B74
:040F5C00C00EF36E62
:100F600000EE00F00E0E01D81200EA6002D0EE6A28
:0C0F7000FCD7F350E9601200EE6AFCD7D9
:01FFF800AC5C
:01FFF900F710
:01FFFA000AFC
:01FFFB00FF06
:01FFFC0063A1
:01FFFD00F80B
:01FFFE000101
:01FFFF00F011
:00000001FF
